:100000000C9446000C9465000C9465000C946500FB
:100010000C9465000C9465000C9465000C946500CC
:100020000C9465000C9465000C9465000C946500BC
:100030000C9465000C9465000C9465000C946500AC
:100040000C9465000C9465000C9465000C9465009C
:100050000C9465000C9465000C9465000C9465008C
:100060000C9465000C9465000C9465000C9465007C
:100070000C9465000C9465000C9465000C9465006C
:100080000C9465000C9465000C94650011241FBE4F
:10009000CFEFD0E1DEBFCDBF11E0A0E0B1E0E6E8F8
:1000A000FAE000E00BBF02C007900D92AC33B1073D
:1000B000D9F711E0ACE3B1E001C01D92A534B1075E
:1000C000E1F70E9480010C9442050C940000882303
:1000D00011F0949A01C0949888B36F70807F862B3A
:1000E00088BB81E0982F9A95F1F7939A8A95F1F75A
:1000F00093988DE08A95F1F708950F931F93082F39
:10010000162F62956F700E946700612F802F0E94EA
:1001100067001F910F91089562E080E00E947D00CA
:1001200081E080933E0180933D0184EF91E001974F
:10013000F1F7089561E080E00E947D0084EF91E096
:100140000197F1F708956EE080E00E947D00089528
:100150006CE080E00E947D0008950E949A000E9459
:100160008C000E94A80008950F931F93182F062F4C
:10017000682F6150023009F4605C606880E00E9482
:100180007D0010933D0100933E011F910F91089552
:1001900080913D018F5F80933D01893244F081E081
:1001A00080933D0180913E018F5F80933E0180915D
:1001B0003E0183301CF081E080933E0108958091E0
:1001C0003D01815080933D01882331F482E080938A
:1001D0003E0188E280933D01089560E180E00E9445
:1001E0007D000E94DF00089564E180E00E947D00B0
:1001F0000E94C800089593988B9A8C9A87B38F6059
:1002000087BB80E197E20197F1F763E080E00E940D
:10021000670081E094E00197F1F763E080E00E94DD
:10022000670081E28A95F1F763E080E00E94670051
:1002300062E080E00E94670068E280E00E947D004A
:1002400066E080E00E947D000E94AD0008951F934B
:10025000182F8A3069F08B301CF48830B9F413C041
:100260008C3019F08D3091F40AC00E94AD0041C06D
:1002700080913E0183301CF48F5F80933E0160913A
:100280003E0181E02AC00E94ED0033C080913C0114
:10029000882321F41B3021F581E012C0813099F4CC
:1002A000612F772767FD70956770707083E0660F28
:1002B000771F8A95E1F7606480E00E947D0082E00C
:1002C00080933C0116C0823059F41B3071F41092B7
:1002D0003C0160913E0180913D010E94B40009C043
:1002E00010320CF417700E94C800612F81E00E9448
:1002F0007D0080E090E01F9108950E9427010895FD
:10030000CFEFD0E1DEBFCDBFBE9ABF9AC6988DE2D7
:1003100091E090934201809341010E94FB0061E0D3
:1003200081E00E94B40080E091E09F938F930E944F
:10033000EE0120E137E20F900F9089E190E0019704
:10034000F1F721503040C9F700E111E0CEE1D1E0F2
:1003500062E082E00E94B4001F930F930E94EE01BE
:1003600020E137E20F900F9089E190E00197F1F7DB
:1003700021503040C9F762E082E00E94B400DF9370
:10038000CF930E94EE01C69A28E833E10F900F90B8
:1003900089E190E00197F1F721503040C9F7C69804
:1003A00020E533EC89E190E00197F1F721503040EE
:1003B000C9F7C79A28E833E189E190E00197F1F79E
:1003C00021503040C9F7C79820E533EC89E190E02F
:1003D0000197F1F721503040C9F7BACFA2E0B0E061
:1003E000E4EFF1E00C941B05FE01379661917191E9
:1003F000FA83E983AF0180914101909142010E940B
:100400000502E2E022960C943705A7E1B0E0EBE0AC
:10041000F2E00C940B058824992454012C017C8B68
:100420006B8B3A01FC0117821682838181FD03C028
:100430008FEF9FEF7EC2CC24DD249E012F5F3F4FC4
:100440003F8B2E8B65C2C0FE48C2832D80538A30FD
:10045000D8F430E3331641F48D85882329F4C3FCA6
:1004600003C0E0E0F1E073C08AE0FD85F802C0015E
:1004700011248053830D8D8787FF02C02FE72D87BE
:10048000C3FC40C22D843EC2960128703070C3FE6A
:1004900005C08D85882311F491E09D87E7E6E3157B
:1004A0006CF1F5E63F160CF068C083E5381609F4E8
:1004B00089C08315BCF09BE2391609F442C093153C
:1004C0004CF0E0E23E1609F440C0F3E23F1609F0BA
:1004D000FCC143C02DE23216E9F13EE2331609F0C9
:1004E000F4C140C083E6381609F44DC083150CF4FE
:1004F00081C098E5391609F0E8C120C0E0E73E1652
:1005000009F4A2C0E3155CF0FCE63F1689F12FE682
:10051000321689F039E6331609F0D7C16BC085E78A
:10052000381609F499C098E7391641F0E3E73E160A
:1005300009F0CBC130C0F8E0F88B8EC020E1288BE9
:100540008BC080E190E0C82AD92AE0E2F0E0CE2A10
:10055000DF2AD8C120E830E00DC080E490E0C82A4E
:10056000D92AD0C1E8E0F0E0CE2ADF2A1D86CAC130
:1005700024E030E0C22AD32AC5C13FE3832E2A9467
:1005800023E6322E30C1F30180802A9422E030E04D
:10059000620E731E28C1F301A081B1814D01232B8E
:1005A00049F0FD856F2F772767FD7095CD010E947B
:1005B000B10418C0FD0101900020E9F73197EA1B52
:1005C000E88B11C0F301808191814C01232B41F014
:1005D000FD856F2F772767FD70950E94A60402C0E6
:1005E0000E949D04888B22E030E0620E731E3889E1
:1005F000231AF9C0C2FE08C0F30180819181A28153
:10060000B38124E030E009C0F30180819181AA2701
:1006100097FDA095BA2F22E030E0620E731E4C01C8
:100620005D01B7FF0CC082E090E0C82AD92AB094DF
:10063000A09490948094811C911CA11CB11CEFEBA0
:10064000FFEFCE22DF2221C020E430E0C22AD32AED
:1006500098E7392E30E1388BC2FE08C0F301808163
:100660009181A281B38124E030E007C0F301808151
:100670009181AA27BB2722E030E0620E731E4C0155
:100680005D018FEC9FEFC822D92285017401FE0124
:100690003196FF87EE87F8898F2E9924AA24BB24F0
:1006A000232D21522D8BC801B701A50194010E9471
:1006B000E9046A301CF03D89630F01C0605DEE857E
:1006C000FF856193FF87EE87C801B701A5019401FB
:1006D0000E94E90479018A0121153105410551057E
:1006E00011F78824992454014E85FE894F1B842ECE
:1006F000C60182739070892B09F02A94C6FE07C048
:100700002889203111F482E001C081E0281AC3FE5B
:1007100012C08D85282F332727FD3095842F9927E8
:10072000821793072CF0E7EFFFEFCE22DF2203C002
:10073000FD85F41BFD87860108701070C3FE03C0A1
:100740002D85221A01C0241AC60180789170892B48
:1007500031F00AC0B20180E290E00E94BC042A9409
:10076000822D8F5F1816B4F3C1FE04C0B2018DE272
:1007700090E00BC0C4FE04C0B2018BE290E005C063
:10078000C5FE05C0B20180E290E00E94BC04C6FE36
:100790000FC0B20180E390E00E94BC043889303180
:1007A00039F4B201832D992787FD90950E94BC04EE
:1007B000D0FC06C00AC0B20180E390E00E94BC04F5
:1007C0002A94822D8F5F1816B4F3012B31F40BC0DD
:1007D000B20180E390E00E94BC048D8581508D873A
:1007E0008F5F1816ACF3F601E078F070FA8BE98BA6
:1007F000C7FE06C00AC0B20180E290E00E94BC04BD
:100800002A94822D8F5F1816B4F3F3E63F1641F455
:10081000B201882D992787FD90950E94BC0445C0A0
:1008200023E73216B1F464017401188909C0F70195
:1008300081917F01B201992787FD90950E94BC04A8
:100840001150A8F74601F8898F0E911C2FEF288BC5
:100850002CC033E5331619F00E851F851FC06401C7
:100860008401F88808C0F8018491B20199270E9498
:10087000BC040F5F1F4FFA94FFEFFF16A1F746016C
:100880002889820E911CF88B10C0F80182918F018B
:10089000B201992787FD90950E94BC042E893F895B
:1008A0000217130791F71F870E8789899A89892B69
:1008B00031F426C0B20180E290E00E94BC042A9488
:1008C000822D8F5F1816B4F31BC0B201832D9927B8
:1008D00087FD90950E94BC0413C095E2391641F43F
:1008E000EAE0E88B22241D8681E0C82ED12C0AC0C4
:1008F000B201832D992787FD90950E94BC0402C008
:10090000CC24DD242B893C892F5F3F4F3C8B2B8BE4
:10091000F201838183FF04C0EB89FC89349003C01A
:10092000EB89FC893080332009F08DCDF20186817E
:100930009781E2E167960C942705FC010590002061
:10094000E9F7809590958E0F9F1F0895FC01059003
:10095000615070400110D8F7809590958E0F9F1FC1
:100960000895FC016150704001900110D8F7809506
:1009700090958E0F9F1F08950F931F93CF93DF9332
:100980008C01EB018B81992781FF1BC082FF0DC079
:100990002E813F818C819D812817390764F4E8817D
:1009A000F9810193F983E88306C0E885F985802FF2
:1009B0000995892B31F48E819F8101969F838E83C7
:1009C00002C00FEF1FEFC801DF91CF911F910F9170
:1009D0000895A1E21A2EAA1BBB1BFD010DC0AA1F80
:1009E000BB1FEE1FFF1FA217B307E407F50720F098
:1009F000A21BB30BE40BF50B661F771F881F991F13
:100A00001A9469F760957095809590959B01AC015B
:100A1000BD01CF0108952F923F924F925F926F9246
:100A20007F928F929F92AF92BF92CF92DF92EF927E
:100A3000FF920F931F93CF93DF93CDB7DEB7CA1BFF
:100A4000DB0B0FB6F894DEBF0FBECDBF09942A882A
:100A5000398848885F846E847D848C849B84AA84D2
:100A6000B984C884DF80EE80FD800C811B81AA815F
:100A7000B981CE0FD11D0FB6F894DEBF0FBECDBF2A
:060A8000ED010895FFCF17
:100A86007374617665626E696365204D4C41420000
:100A960064656D6F2061706C696B61636500202011
:100AA60020202020202020202020202000000000C0
:0C0AB60002000000007D010000000000B4
:00000001FF
